:020000020000FC
:1000000000C000C00FED0DBF09E109B978D050E084
:100010002AE351D020E24FD020E24DD052D01F32FF
:10002000B1F01F3319F11032A9F11D3041F1113235
:10003000F9F0153279F01F7D123509F1173509F104
:10004000113459F11135E9F21D3449F1E1CF5A95D6
:1000500090D0DECF40D04ED0F0E0E52F30817AD086
:1000600020E229D0549A5F9BF5CFD2CF48D0D0CF91
:10007000F3E0EEE534D0A89508E001BDFFCF79D0DC
:10008000C7CFF3E0E2E52BD06ED0F0E0E52F308370
:1000900070D0BECF53956DD0BBCF74D0B9CF1BD02D
:1000A00029D0F0E0E52F30814FD020E204D0549ADF
:1000B0005F9BF5CFADCF539A5D9BFDCF2CB9539885
:1000C0000895549A5F9BFDCF1CB154980895F9DFB1
:1000D000212FF1DF0895F3E0EEE401D00895C895F3
:1000E000002021F0202DE7DF3196F9CF0895F7DFCA
:1000F000F2DF0895352F28D020E2DDDF0895EBDF11
:10010000EADFF1E0EEE8F3DF0895F3E0E2E4E7DFB1
:100110000895432F4695469546954695405D4A334A
:1001200008F0495F3F70305D3A3308F0395F089559
:1001300046FD475F4F7036FD375F3F70440F440FF9
:10014000440F440F342B0895E4DF242FB4DF232F12
:10015000B2DF089508E020E3331F08F421E3ABDFAA
:100160000A95C9F70895B3DF412FB1DF312FE0DFE2
:100170000895B1DFBFDFF0E0E52F3081E5DF20E259
:100180009ADF0895C2DFEFDF532FF3DF0895323394
:100190003133206D6F6E69746F72202032303032CF
:1001A0002E30322E303120562020202020202020BA
:1001B0002020202020204469636B204361707065FB
:1001C0006C730A0D41203D20736574206164647274
:1001D000657373200A0D57203D207772697465207E
:1001E0000A0D52206F72203C43523E203D2073681E
:1001F0006F77206D656D6F727920636F6E74656EB9
:1002000074732061742063757272656E742061640A
:100210006472657373200A0D3C73706163653E20E0
:100220003D20696E6372656D656E742063757272D0
:10023000656E74206164647265737320616E6420FE
:10024000646973706C6179200A0D2F203D2064650C
:100250006372656D656E742063757272656E74206D
:100260006164647265737320616E64206469737085
:100270006C6179200A0D4D203D206D6F6E69746FA1
:1002800072206461746120756E74696C206B65798D
:1002900020707265737365640A0D25203D206D6FB3
:1002A0006E69746F72206461746120616E64207382
:1002B000686F7720696E2062696E617279200A0D1D
:1002C0003F203D2074797065206F70656E696E67A0
:1002D0002073637265656E2E0A0D51203D20726594
:1002E0007374617274206669726D776172650A0D4C
:1002F00021203D20726573657420636869700A0D62
:10030000416C6C206164647265737320616E64205B
:10031000646174612076616C75657320617265201B
:1003200068657861646563696D616C20616E6420E5
:10033000617265206279746520776964652E0A0DA3
:100340000000416464726573733A202000000A0D56
:1003500000006E657720646174613A200000486196
:100360007264776172652072657365742076696165
:10037000207761746368646F6720696E697469616E
:060380007465642E00000C
:00000001FF
